:100000005BEF0BF0FFFFFFFF0000000012000F0E80
:100010000B6EFF0E0A6E0B2E01D003D00A2EFED7F8
:10002000FAD73E0E0A6E0A2EFED700001200210EED
:100030000A6E0A2EFED7120000018551390807E327
:10004000300E855D04E3010E006E28EF00F0006ABB
:100050001200000100500402F4CF09F0F3CF08F0C1
:1000600001500502F4CF0BF0F3CF0AF00050050267
:10007000F3500926F4500A22E86A0B2201500402C8
:10008000F3500926F4500A22E86A0B2205AE4DEF20
:1000900000F000500A5C01500B5801AE54EF00F024
:1000A00004500A5C05500B5808C000F009C001F06C
:1000B0000AC002F00BC003F0120000010B6A0A6ACA
:1000C000096A086A0E6A033408360450085E05504F
:1000D000D8A0053C095E0650D8A0063C0A5E075031
:1000E000D8A0073C0B5EE86AD8A0010E0E5E03366E
:1000F000070E0C6E0334083609360A360B360E36F8
:10010000045003A097EF00F0085E0550D8A0053C0E
:10011000095E0650D8A0063C0A5E0750D8A0073CEE
:100120000B5EE86AD8A0010E0E5EA8EF00F008266C
:100130000550D8B0053C09260650D8B0063C0A2622
:100140000750D8B0073C0B26E86AD8B0010E0E263F
:1001500003360C2E7AEF00F00234083609360A36E0
:100160000B360E36045003A0C9EF00F0085E0550B0
:10017000D8A0053C095E0650D8A0063C0A5E075090
:10018000D8A0073C0B5EE86AD8A0010E0E5EDAEF3D
:1001900000F008260550D8B0053C09260650D8B016
:1001A000063C0A260750D8B0073C0B26E86AD8B0B0
:1001B000010E0E260236070E0C6E02340836093682
:1001C0000A360B360E36045002A0FAEF00F0085E35
:1001D0000550D8A0053C095E0650D8A0063C0A5E32
:1001E0000750D8A0073C0B5EE86AD8A0010E0E5E4F
:1001F0000BEF01F008260550D8B0053C0926065043
:10020000D8B0063C0A260750D8B0073C0B26E86A4F
:10021000D8B0010E0E2602360C2EDDEF00F00134B0
:10022000083609360A360B360E36045002A02CEF7B
:1002300001F0085E0550D8A0053C095E0650D8A024
:10024000063C0A5E0750D8A0073C0B5EE86AD8A0BF
:10025000010E0E5E3DEF01F008260550D8B0053CBA
:1002600009260650D8B0063C0A260750D8B0073CED
:100270000B26E86AD8B0010E0E260136070E0C6E6A
:100280000134083609360A360B360E36045001A002
:100290005DEF01F0085E0550D8A0053C095E0650F0
:1002A000D8A0063C0A5E0750D8A0073C0B5EE86A5F
:1002B000D8A0010E0E5E6EEF01F008260550D8B0F2
:1002C000053C09260650D8B0063C0A260750D8B08F
:1002D000073C0B26E86AD8B0010E0E2601360C2E1C
:1002E00040EF01F00034083609360A360B360E3678
:1002F000045001A08FEF01F0085E0550D8A0053C26
:10030000095E0650D8A0063C0A5E0750D8A0073CFC
:100310000B5EE86AD8A0010E0E5EA0EF01F0082681
:100320000550D8B0053C09260650D8B0063C0A2630
:100330000750D8B0073C0B26E86AD8B0010E0E264D
:100340000036070E0C6E0034083609360A360B36B6
:100350000E36045000A0C0EF01F0085E0550D8A092
:10036000053C095E0650D8A0063C0A5E0750D8A09E
:10037000073C0B5EE86AD8A0010E0E5ED1EF01F0DB
:1003800008260550D8B0053C09260650D8B0063CD2
:100390000A260750D8B0073C0B26E86AD8B0010EF1
:1003A0000E2600360C2EA3EF01F000B0E6EF01F0B0
:1003B000045008260550D8B0053C09260650D8B090
:1003C000063C0A260750D8B0073C0B2612001550F1
:1003D000161000E015C0E9FF16C0EAFF00018553C2
:1003E00000E0EF96EF9EEF9CEF9AEF98EF9485BFB9
:1003F000EF8E85BDEF8C85BBEF8A85B9EF881750EE
:10040000010A03E1EF9406EF02F0EF84EF8604ECBB
:1004100000F00001855300E0EF96EF9EEF9CEF9A0D
:10042000EF98EF9485B7EF8E85B5EF8C85B3EF8AA3
:1004300085B1EF881750010A03E1EF9421EF02F034
:10044000EF84EF8604EC00F0EF961750010A03E109
:1004500007EC00F002D017EC00F012006E0E5B6E9D
:100460006F0E5C6E6E0E5D6E2D0E5E6E660E5F6EB6
:100470006C0E0001606F6F0E616F610E626F740E23
:10048000636F200E646F700E656F720E666F690E7B
:10049000676F6E0E686F740E696F660E6A6F6B6BB6
:1004A000280E6C6F6E0E6D6F750E6E6F6C0E6F6F2B
:1004B0006C0E706F290E716F726B7A6B7B6B786B41
:1004C000796B56C000F057C001F058C002F0010E21
:1004D0005626000E5722582200C0F6FF01C0F7FF33
:1004E00002C0F8FF0900F5CF00F000C075F000521F
:1004F000D8B42CEF0AF000017551250A0BE054C066
:10050000E1FF55C0E2FF75C0E6FF544A552A7A4B19
:100510007B2BD7D70001766B776B786B796B28D004
:1005200000017887010E5626000E572258225ED011
:1005300000017881010E5626000E5722582256D00F
:1005400000017883010E5626000E572258224ED005
:1005500000017987010E5626000E5722582246D0F8
:1005600000017885010E5626000E572258223ED0F3
:1005700056C0F6FF57C0F7FF58C0F8FF0900F5CF87
:1005800080F0000180512D0ACBE056C0F6FF57C025
:10059000F7FF58C0F8FF0900F5CF80F08051200A1E
:1005A000C7E056C0F6FF57C0F7FF58C0F8FF090074
:1005B000F5CF80F080512B0AC3E056C0F6FF57C03C
:1005C000F7FF58C0F8FF0900F5CF80F08051230AEB
:1005D000BFE056C0F6FF57C0F7FF58C0F8FF09004C
:1005E000F5CF80F08051300ABBE001D098D70001F0
:1005F00078B37891000178B7789556C0F6FF57C068
:10060000F7FF58C0F8FF0900F5CF00F0000E016EAB
:1006100000C085F01CEC00F0005238E00001766B61
:10062000776B000176C000F077C001F00A0E046E0F
:10063000000E056E29EC00F056C0F6FF57C0F7FF1C
:1006400058C0F8FF0900F5CF80F080510024766F84
:10065000000E0120776F300E765F000E775B010E83
:100660005626000E5722582256C0F6FF57C0F7FFF5
:1006700058C0F8FF0900F5CF00F0000E016E00C071
:1006800085F01CEC00F00052CCE136D056C0F6FFED
:1006900057C0F7FF58C0F8FF0900F5CF80F0000100
:1006A00080512A0A29E159C0E9FF5AC0EAFFEECF7A
:1006B00000F0EECF01F000C0E9FF01C0EAFFEECF8D
:1006C00076F0EECF77F059C0E9FF5AC0EAFFEECFDF
:1006D00000F0EECF01F0020E0026000E012259C0FC
:1006E000E1FF5AC0E2FF00C0E6FF01C0E6FF010ED5
:1006F0005626000E5722582256C0F6FF57C0F7FF65
:1007000058C0F8FF0900F5CF80F0000180512E0A93
:1007100074E1010E5626000E5722582256C0F6FFED
:1007200057C0F7FF58C0F8FF0900F5CF80F080519F
:100730002A0A2AE159C0E9FF5AC0EAFFEECF00F0C9
:10074000EECF01F000C0E9FF01C0EAFFEECF73F089
:10075000EECF74F059C0E9FF5AC0EAFFEECF00F0C7
:10076000EECF01F0020E0026000E012259C0E1FF7B
:100770005AC0E2FF00C0E6FF01C0E6FF010E5626A8
:10078000000E5722582237D00001736B746B56C08D
:10079000F6FF57C0F7FF58C0F8FF0900F5CF00F08B
:1007A000000E016E00C085F01CEC00F0005223E04A
:1007B00073C000F074C001F00A0E046E000E056EE6
:1007C00029EC00F056C0F6FF57C0F7FF58C0F8FFFD
:1007D0000900F5CF80F080510024736F000E0120D6
:1007E000746F300E735F000E745B010E5626000EA0
:1007F00057225822CCD7000103D00001736B746BD1
:1008000056C000F057C001F058C002F0010E562645
:10081000000E5722582200C0F6FF01C0F7FF02C0A9
:10082000F8FF0900F5CF75F0FED07AC000F07BC06C
:1008300001F0120000017889E3D75B0E00017C6FA4
:10084000000E7D6F736B746B2DD00001788D27D1F6
:1008500026D10001788B0001788F21D159C0E9FFA2
:100860005AC0EAFFEECF00F0EECF01F000C0E9FF82
:1008700001C0EAFFEECF7CF0EECF7DF059C0E9FF7A
:100880005AC0EAFFEECF00F0EECF01F0020E0026D4
:10089000000E012259C0E1FF5AC0E2FF00C0E6FF8E
:1008A00001C0E6FF000E00017D1902E1000E7C1977
:1008B00005E16C0E00017C6F000E7D6F00017E6B08
:1008C0007F6B00017E517C25E96E7F517D21EA6EB0
:1008D000EECF00F0005203E07E4B7F2BF2D70001F9
:1008E000735174110AE07F51745D02E17E51735DB2
:1008F00004E273C07EF074C07FF0000177517F5D29
:1009000002E176517E5D06E200017E51765F7F5105
:10091000775B03D00001766B776B000178B717D057
:1009200076C000F077C001F0010E0001765F000E86
:10093000775B005001100BE054C0E1FF55C0E2FFAF
:10094000200EE66E544A552A7A4B7B2BE9D77EC09F
:1009500000F07FC001F0010E00017E5F000E7F5BA2
:100960000050011013E07CC0E9FF7DC0EAFFEECF2C
:1009700000F054C0E1FF55C0E2FF00C0E6FF544A5A
:10098000552A7C4B7D2B7A4B7B2BE1D7000178A736
:1009900017D076C000F077C001F0010E0001765F3D
:1009A000000E775B005001100BE054C0E1FF55C012
:1009B000E2FF200EE66E544A552A7A4B7B2BE9D78C
:1009C00080D559C0E9FF5AC0EAFFEECF00F0EECF64
:1009D00001F000C0E9FF01C0EAFFEECF75F059C099
:1009E000E9FF5AC0EAFFEECF00F0EECF01F0020EB1
:1009F0000026000E012259C0E1FF5AC0E2FF00C0EC
:100A0000E6FF01C0E6FF750E00017C6F000E7D6FF2
:100A1000010E7E6F000E7F6F62D7C00E000178134B
:100A2000000E79133CD000017551000AD8B4FDD6F0
:100A300075516C0AD8B4FED67551450AD8B4FDD6A6
:100A40007551660AD8B4F9D67551650AD8B4F5D689
:100A50007551670AD8B4F1D675516F0AD8B4F5D676
:100A60007551640AD8B4F4D67551690AD8B4F0D671
:100A70007551700AD8B4EDD67551580AD8B4E9D674
:100A80007551780AD8B4E7D67551730AD8B4E6D64A
:100A90007551630A96E07551750ABFE0B4D7C00E70
:100AA00000017815806F79C081F0000E8117000E6B
:100AB000811902E1000E8019D8A485D0000178A91F
:100AC00029D059C0E9FF5AC0EAFFEECF00F0EECFBF
:100AD00001F000C0E9FF01C0EAFFEECF7CF0EECFED
:100AE0007DF0EECF7EF0EECF7FF059C0E9FF5AC027
:100AF000EAFFEECF00F0EECF01F0040E0026000E6C
:100B0000012259C0E1FF5AC0E2FF00C0E6FF01C068
:100B1000E6FF2FD059C0E9FF5AC0EAFFEECF00F040
:100B2000EECF01F000C0E9FF01C0EAFFEECF7CF09C
:100B3000EECF7DF0000E00017DBFFF0E7E6F7F6F58
:100B4000000E7DBFFF0E7E6F7F6F59C0E9FF5AC058
:100B5000EAFFEECF00F0EECF01F0020E0026000E0D
:100B6000012259C0E1FF5AC0E2FF00C0E6FF01C008
:100B7000E6FF800E00017F19006E800E005C08E128
:100B8000000E7E5D05E1000E7D5D02E1000E7C5DE4
:100B900019E2030E00017813000E7913006A016A4E
:100BA000026A036A7C51005E7D51015A7E51025AED
:100BB0007F51035A00C07CF001C07DF002C07EF07E
:100BC00003C07FF057D0000178A929D059C0E9FFB0
:100BD0005AC0EAFFEECF00F0EECF01F000C0E9FF0F
:100BE00001C0EAFFEECF7CF0EECF7DF0EECF7EF0DD
:100BF000EECF7FF059C0E9FF5AC0EAFFEECF00F018
:100C0000EECF01F0040E0026000E012259C0E1FFD4
:100C10005AC0E2FF00C0E6FF01C0E6FF2BD059C07A
:100C2000E9FF5AC0EAFFEECF00F0EECF01F000C0BE
:100C3000E9FF01C0EAFFEECF7CF0EECF7DF0000EC1
:100C400000017E6F7F6F000E7E6F7F6F59C0E9FFDE
:100C50005AC0EAFFEECF00F0EECF01F0020E002600
:100C6000000E012259C0E1FF5AC0E2FF00C0E6FFBA
:100C700001C0E6FF000E0001741902E1000E7319B5
:100C800011E1000E006E00017F1908E100507E198D
:100C900005E100507D1902E17C51000A03E10001E9
:100CA000734B742BC00E00017815006E00C084F0E9
:100CB000C3D0010E0001756F000175510A0A39E0B9
:100CC000020E046E75C000F0000E016E026E036E1F
:100CD000045007E000360090013602360336FF0F5D
:100CE000F8D78C0E0026170E0122000E022200C03B
:100CF000F6FF01C0F7FF02C0F8FF0900F5CF80F052
:100D00000900F5CF81F00900F5CF82F00900F5CF99
:100D100083F0000183517F5D08E182517E5D05E132
:100D200081517D5D02E180517C5D03E30001752B03
:100D3000C3D792D0010E0001756F00017551080AEA
:100D400039E0020E046E75C000F0000E016E026EF6
:100D5000036E045007E00036009001360236033679
:100D6000FF0FF8D7B40E0026170E0122000E022244
:100D700000C0F6FF01C0F7FF02C0F8FF0900F5CF81
:100D800080F00900F5CF81F00900F5CF82F009006D
:100D9000F5CF83F0000183517F5D08E182517E5DD4
:100DA00005E181517D5D02E180517C5D03E300013D
:100DB000752BC3D751D0010E0001756F000175511D
:100DC0000C0A39E0020E046E75C000F0000E016ED0
:100DD000026E036E045007E00036009001360236C2
:100DE0000336FF0FF8D7D40E0026170E0122000E8F
:100DF000022200C0F6FF01C0F7FF02C0F8FF0900A1
:100E0000F5CF80F00900F5CF81F00900F5CF82F031
:100E10000900F5CF83F0000183517F5D08E1825125
:100E20007E5D05E181517D5D02E180517C5D03E3E2
:100E30000001752BC3D710D000018451000AD8B42B
:100E400038D78451C00AD8B434D78451800AD8B472
:100E500071D78451400AAFE0800E006E800E000111
:100E60007419005C02E17351755D03E273C075F0A3
:100E70000FD0800E00017419006E800E005C02E13C
:100E80007551735D05E275C073F0000E0001746F5B
:100E90000001765177110FE0030E7815006E79C0CE
:100EA00001F0000E01160050011005E0010E0001D6
:100EB000765F000E775B800E00017419006E800E65
:100EC0007719005C02E17651735D06E2000173510F
:100ED000765F7451775B03D00001766B776BC40E3D
:100EE00000017815806F7951080B816F8151080AD4
:100EF00002E1400E801909E100017651771104E00A
:100F0000010E765F000E775B20D0C00E00017815D1
:100F1000806F7951080B816F8151080A02E1800EC0
:100F2000801913E1800E006E800E00017719005CBD
:100F300002E17651020806E2020E0001765F000E21
:100F4000775B03D00001766B776B000178A574D0D6
:100F500078A31BD0010E7815006E79C001F0000E49
:100F600001160050011003E02D0E006E02D02B0E72
:100F7000006E54C0E1FF55C0E2FF00C0E6FF544AD6
:100F8000552A00017A4B7B2B40D0010E00017815C9
:100F9000006E79C001F0000E0116005001100BE048
:100FA00054C0E1FF55C0E2FF200EE66E544A552AB8
:100FB0007A4B7B2B2AD0C00E00017815806F7951B7
:100FC000080B816F8151080A02E1800E80191DE132
:100FD00054C0E1FF55C0E2FF300EE66E544A552A78
:100FE00000017A4B7B2B78AB03D0580E006E02D0F9
:100FF000780E006E54C0E1FF55C0E2FF00C0E6FF6E
:10100000544A552A00017A4B7B2B00017651771107
:1010100012E054C0E1FF55C0E2FF300EE66E544AC4
:10102000552A00017A4B7B2B010E765F000E775B11
:1010300076517711EEE18ED000017651771114E0F0
:1010400078B712D054C0E1FF55C0E2FF200EE66E23
:10105000544A552A00017A4B7B2B010E765F000E15
:10106000775B76517711EEE1000178A31BD0010E7A
:101070007815006E79C001F0000E011600500110C5
:1010800003E02D0E006E02D02B0E006E54C0E1FF67
:1010900055C0E2FF00C0E6FF544A552A00017A4BD2
:1010A0007B2B15D0010E00017815006E79C001F080
:1010B000000E0116005001100AE054C0E1FF55C0B7
:1010C000E2FF200EE66E544A552A7A4B7B2BC00E67
:1010D00000017815806F7951080B816F8151080AE2
:1010E00002E1400E80190CE154C0E1FF55C0E2FF5F
:1010F000300EE66E544A552A00017A4B7B2B2AD0DB
:10110000C00E00017815806F7951080B816F8151F5
:10111000080A02E1800E80191DE154C0E1FF55C0AC
:10112000E2FF300EE66E544A552A00017A4B7B2BC3
:1011300078AB03D0580E006E02D0780E006E54C00B
:10114000E1FF55C0E2FF00C0E6FF544A552A000106
:101150007A4B7B2B800E006E800E00017419005CB0
:1011600002E17351755D0CE254C0E1FF55C0E2FF2E
:10117000300EE66E544A552A00017A4B7B2BEAD793
:1011800073C000F074C001F0010E0001735F000E27
:10119000745B00500110D8B441D1C00E7815006EB8
:1011A00000C080F021D1020E046E73C000F074C044
:1011B00001F0000E000174BFFF0E026E036E0450BA
:1011C00007E000360090013602360336FF0FF8D7ED
:1011D0008C0E0026170E0122000E022200C0F6FF20
:1011E00001C0F7FF02C0F8FF0900F5CF04F00900C5
:1011F000F5CF05F00900F5CF06F00900F5CF07F0AF
:101200007CC000F07DC001F07EC002F07FC003F022
:101210005DEC00F00A0E046E000E056E066E076EA1
:101220005DEC00F008C000F009C001F00AC002F057
:101230000BC003F0300E0024756FE5D078AB4CD0B6
:10124000020E046E73C000F074C001F0000E74BF93
:10125000FF0E026E036E045007E000360090013668
:1012600002360336FF0FF8D7B40E0026170E012200
:10127000000E022200C0F6FF01C0F7FF02C0F8FF17
:101280000900F5CF04F00900F5CF05F00900F5CF0E
:1012900006F00900F5CF07F07CC000F07DC001F03A
:1012A0007EC002F07FC003F05DEC00F00F0E001670
:1012B000000E011602160316040E0026180E012257
:1012C000000E022200C0F6FF01C0F7FF02C0F8FFC7
:1012D0000900F5CF75F04BD0020E046E73C000F01C
:1012E00074C001F0000E74BFFF0E026E036E045056
:1012F00007E000360090013602360336FF0FF8D7BC
:10130000B40E0026170E0122000E022200C0F6FFC6
:1013100001C0F7FF02C0F8FF0900F5CF04F0090093
:10132000F5CF05F00900F5CF06F00900F5CF07F07D
:101330007CC000F07DC001F07EC002F07FC003F0F1
:101340005DEC00F00F0E0016000E011602160316DB
:10135000160E0026180E0122000E022200C0F6FF13
:1013600001C0F7FF02C0F8FF0900F5CF75F04BD0C0
:10137000020E046E73C000F074C001F0000E74BF62
:10138000FF0E026E036E045007E000360090013637
:1013900002360336FF0FF8D7D40E0026170E0122AF
:1013A000000E022200C0F6FF01C0F7FF02C0F8FFE6
:1013B0000900F5CF04F00900F5CF05F00900F5CFDD
:1013C00006F00900F5CF07F07CC000F07DC001F009
:1013D0007EC002F07FC003F05DEC00F0070E001449
:1013E000756F300E75270FD08051000AD8B4DBD648
:1013F0008051C00AD8B4D7D68051800AD8B41ED73D
:101400008051400AB5E054C0E1FF55C0E2FF75C00D
:10141000E6FF544A552A7A4B7B2BB2D678A71AD0CE
:10142000800E006E800E7719005C02E17651000894
:1014300011E254C0E1FF55C0E2FF200EE66E544AAF
:10144000552A7A4B7B2B010E765F000E775B765127
:101450007711EFE161EF02F07AC000F07BC001F09C
:101460001200176A54C085F0E7EC01F0010E176E08
:10147000120047C015F048C016F047C0E1FF48C051
:10148000E2FFE66A47C015F048C016F0110EE126EB
:10149000E76A120EE15E07EC00F0E78AE788E7866C
:1014A00004EC00F0E79607EC00F0E78AE788E786AF
:1014B00004EC00F0E79617EC00F017EC00F0E78A78
:1014C000E788E78604EC00F0E79607EC00F0E78A8F
:1014D000E798E78604EC00F0E79617EC00F0E78A5F
:1014E000E798E78604EC00F0E796E78EE79CE7864E
:1014F00004EC00F0E79617EC00F0000EE76EE786CC
:1015000004EC00F0E796E78EE78CE78AE788E78649
:1015100004EC00F0E79617EC00F0000EE76EE786AB
:1015200004EC00F0E796E788E78604EC00F0E79625
:1015300007EC00F0000EE76EE78604EC00F0E7969B
:10154000E78CE78AE78604EC00F0E79617EC00F0FA
:10155000010E176E12000FD0800E476E19D0C00E0C
:10156000476E16D0940E476E13D0D40E476E10D02F
:10157000800E476E0DD04750010AEEE04750020A38
:10158000EEE04750030AEEE04750040AEEE0F0D7E1
:101590004804006E4750002600C047F000C085F0A8
:1015A000E7EC01F0176A4B6A4C6A4B504924E96E2C
:1015B0004C504A20EA6EEECF00F000520DE04B5046
:1015C0004924E96E4C504A20EA6EEECF85F0E7ECF4
:1015D00001F04B4A4C2AE9D7010E176E12004C0E4F
:1015E000526E000E536E47C054F048C055F049C0CB
:1015F00056F04AC057F04BC058F0520E596E000ECC
:101600005A6E2EEC02F000C050F001C051F00050B4
:101610004724E16E01504820E26EE66A50C000F0B7
:1016200051C001F01200496A4A6A49504724E96EE4
:101630004A504820EA6EEECF00F000520DE04950CB
:101640004724E96E4A504820EA6EEECF54F031EC60
:101650000AF0494A4A2AE9D71200490E186E6E0E5E
:10166000196E2D0E1A6E430E1B6E690E1C6E720ED5
:101670001D6E630E1E6E750E1F6E690E206E740E4B
:10168000216E200E226E500E236E490E246E430EE4
:10169000256E4C0E266E6F0E276E610E286E640E40
:1016A000296E650E2A6E720E2B6E2C6A180E2D6E28
:1016B000000E2E6E12002DEC0BF0436A446A456A50
:1016C000466A0E0EC16E936A956A810E476E0F0EC2
:1016D000486E39EC0AF0010E0001856FE7EC01F06D
:1016E0000C0E0001856FE7EC01F0010E476E010E54
:1016F000486E2DC049F02EC04AF0ABEC0AF0C00E87
:101700000001856FE7EC01F02F0E476E000E486E6A
:10171000280E496E180E4A6E000E4B6E43C04CF0F8
:1017200044C04DF045C04EF046C04FF0EFEC0AF01B
:10173000010E4326000E4422452246222F0E476EFC
:10174000000E486E13EC0BF0020E0C6EFF0E0B6ECB
:10175000FF0E0A6E0C2E01D007D00B2E01D003D045
:101760000A2EFED7FAD7F6D7060E0B6EFF0E0A6EBC
:101770000B2E01D003D00A2EFED7FAD70A0E0A6E1E
:101780000A2EFED70000837EBAD7FFD701000000E3
:101790000A00000064000000E803000010270000B9
:1017A000A086010040420F008096980000E1F505F8
:1017B00000CA9A3B01000000100000000001000078
:1017C00000100000000001000000100000000001F7
:1017D00000000010010000000800000040000000B0
:1017E0000002000000100000008000000000040063
:1017F0000000200000000001000000080000004080
:101800000000000030313233343536373839414248
:101810004344454600FF30313233343536373839AA
:1018200061626364656600FF256C6400FFFFFFFF73
:020000040030CA
:0E000000FFFAFFFEFFFFFBFFFFFFFFFFFFFF0A
:00000001FF
